:020000000528D1
:10000800090083160730850000308100073096000C
:1000180070308F007F30900000309F0083120730CF
:100028009900043092000000A3010508FF3A07393F
:10003800031D1828A30B19288B1505080B1063003E
:1000480026201728851C2D28051C3228051D372831
:10005800262839207730851C88303B28392099306C
:10006800051CAA303B28BB303B2855306528A10029
:10007800A0001030522012305220210847202108B9
:10008800FF3A47200800A0000830A30009302018D4
:100098001A305220A00CA30B4A280800A2005E20A8
:1000A800A20B532805165E200512000085165E2057
:1000B800851208005030A40000000000A40B60283E
:1000C8000800A400A500A600A60B6828A50B6728B1
:0600D800A40B66280800DD
:02400E00E4309C
:00000001FF
